:10000000292890309D00062810309D009C01920107
:10001000180D9C0D920D1E089C021A08031C1A0F45
:10002000920203181A281E089C071A0803181A0FB0
:10003000920703109F0D980D9D031F301D05031D92
:1000400008289D1B2728180892001F0808001C0874
:1000500008008316FF3085001F308600583081006D
:10006000043095009601970119309B0083120F30E0
:1000700006058F0007300F0299008F011908031938
:100080008F0A0F088C0003195128FE3015029000CA
:1000900016089100031C91038F01911B8F0A0F0812
:1000A0008C000C0803195F28023015079000160811
:1000B00091000318910A1108960010089500831208
:1000C0000F3006058C000B300C0299008C011908CA
:1000D00003198C0A0C088F0003197B281508003CB3
:1000E00090009101031C9103160891028C01911B51
:1000F0008C0A0C088F000F0803198928023015029A
:10010000900016089100031C910311089600100836
:10011000950019301B028F0099010F080319990AE5
:1001200019088C000319A12883120F3006058F00CF
:100130000D300F0299008F01190803198F0A0F085B
:100140008C000C080319A828970A17039B01B328F1
:1001500019301B028C008F018C1B8F0A0F080319AA
:10016000B3289B0A1B031508FE3C90009101031C59
:100170009103160891021008A00017089F0098012B
:10018000971B980303309E009A01012093001208E8
:1001900094008C011308140403198C0A0C08031929
:1001A000002997018E0105300E028C008F018C1BF7
:1001B0008F0A0F0803190029831286018D01150883
:1001C0000D0293009101031C91038F01031C8F0A00
:1001D0000F080319EE288D0A0D03DF288312E03083
:1001E00086008D0120080D028F01031C8F0A0F0865
:1001F0000319FD288D0A0D03F2288E0A0E03D32859
:1002000017089F009801971B980303309E009A01DE
:1002100001209300120891009303031C91038C01A9
:100220001308110403198C0A0C08031946298E01BE
:1002300005300E028C008F018C1B8F0A0F080319EA
:1002400046298312C03086008D0115080D029300E7
:100250009401031C94038F01031C8F0A0F080319D8
:1002600034298D0A0D0325298312E03086008D0183
:1002700020080D028F01031C8F0A0F080319432960
:100280008D0A0D0338298E0A0E03182917089F00BE
:100290009801971B980303309E009A010120930058
:1002A00012089400023013029300031C940392017D
:1002B000130814040319920A12080319652A8312F9
:1002C000E0308600031103140430060592008C010F
:1002D000120803198C0A0C0803196F296300831292
:1002E000031103140830060592008C01120803194B
:1002F0008C0A0C0803194C2A831286018E01803067
:100300000E028C01031C8C0A0C08031996298D011E
:10031000FF300D028C01031C8C0A0C080319932971
:100320008D0A0D0388298E0A0E037F298312C0309F
:1003300086008E0180300E028C01031C8C0A0C0892
:100340000319B1298D01FF300D028C01031C8C0AA9
:100350000C080319AE298D0A0D03A3298E0A0E037A
:100360009A298312803086008E0180300E028C0123
:10037000031C8C0A0C080319CC298D01FF300D02D7
:100380008C01031C8C0A0C080319C9298D0A0D0362
:10039000BE298E0A0E03B5298312A03086008E0175
:1003A00080300E028C01031C8C0A0C080319E7290B
:1003B0008D01FF300D028C01031C8C0A0C080319FF
:1003C000E4298D0A0D03D9298E0A0E03D029831240
:1003D000203086008E0180300E028C01031C8C0AB6
:1003E0000C080319022A8D01FF300D028C01031C39
:1003F0008C0A0C080319FF298D0A0D03F4298E0AB3
:100400000E03EB298312603086008E0180300E02CD
:100410008C01031C8C0A0C0803191D2A8D01FF3066
:100420000D028C01031C8C0A0C0803191A2A8D0A70
:100430000D030F2A8E0A0E03062A8312403086000F
:100440008E0180300E028C01031C8C0A0C080319EB
:10045000382A8D01FF300D028C01031C8C0A0C0818
:100460000319352A8D0A0D032A2A8E0A0E03212A22
:100470008312E030860083161F30860083120F300F
:10048000060592000F3012028C0092018C1B920A1A
:100490001208031D4C2A7C298E0105300E029200A1
:1004A0008C01921B8C0A0C080319652A8D0180307F
:1004B0000D029201031C920A12080319622A8D0A86
:0E04C0000D03572A8E0A0E034D2A3628662A8F
:084000000100020003000400AE
:02400E00F23F7F
:00000001FF
